:103C00000C94381E0C94551E0C94551E0C94551E85
:103C10000C94551E0C94551E0C94551E0C94551E58
:103C20000C94551E0C94551E0C94551E0C94551E48
:103C30000C94551E0C94551E0C94551E0C94551E38
:103C40000C94551E0C94551E0C94551E0C94551E28
:103C50000C94551E0C94551E0C94551E0C94551E18
:103C60000C94551E0C94551E0C94551E0C94551E08
:103C700011241FBECFEFD4E0DEBFCDBF11E0A0E026
:103C8000B1E0ECEAFFE302C005900D92A230B1076B
:103C9000D9F711E0A2E0B1E001C01D92A838B10748
:103CA000E1F70E94C91E0C94D41F0C94001ECF9300
:103CB000DF93EC01A0910401B091050183E0FD01C7
:103CC00080935700E89507B600FCFDCF109287015E
:103CD00071E014C0262F30E0FE01E20FF31F518186
:103CE00040E0808190E0842B952BF9010C017093CA
:103CF0005700E89511246E5F6093870160918701FA
:103D000067FFE8CF85E0FD0180935700E89507B68F
:103D100000FCFDCFDF91CF910895E199FECF8FEFA9
:103D200091E09FBB8EBBE09A8DB3882319F0E0E051
:103D3000FCE3099581E180935700E895E0E0F0E02D
:103D4000099508958CB95E9BFECF5E9A08955F9B9E
:103D5000FECF8CB10895FC0170E880E090E0A1E214
:103D6000B0E1508140E08427952768E09C01220F54
:103D7000331F97FF02C02A273B276150C901B1F7C3
:103D8000715011F03196EDCF3093860120930301ED
:103D90000895BF92CF92DF92EF92FF920F931F93FD
:103DA000F89414BE28E10FB6F89421BD11BC0FBEE3
:103DB00085E39CE09BBD8ABD1FBC8DE08EBDA39AB0
:103DC0001BB82AB986E880BD10BC83E389B910927C
:103DD00003011AE008E008B606FE0EC088B780644A
:103DE00088BF809103018130D1F085B3802785BBE6
:103DF000115011F40E948D1E5F9BEDCF8CB120916C
:103E00000301E22FF0E0E050FF4F9081891721F489
:103E10002F5F20930301DFCF10920301DCCFE199E4
:103E2000FECF8FEF91E09FBB8EBB81E08DBB0FB6C5
:103E3000F894E29AE19A0FBE1EE1E3E4FE2E08E058
:103E400008B606FE0EC088B7806488BFFCB85E9BCB
:103E5000FECF5E9A85B3802785BB115011F40E9476
:103E60008D1E5F9BEDCF8CB1813051F71EBC10923F
:103E70000201109205011092040110E0EE2475E198
:103E8000D72E66E0B62E58E0C52EE3945F9BFECF9A
:103E90009CB1909386015F9BFECF8CB180958093FF
:103EA0000301E91609F050C0E81609F04DC09091E1
:103EB0000201292F20585F9BFECF8CB1E92FF0E043
:103EC000EA5FFE4F80839F5F9217A9F790930201EC
:103ED0005F9BFECF0CB15F9BFECFFCB0892F90E0C3
:103EE0008A579F4F0E94AB1E80918601081741F5AB
:103EF00080910301F81621F580910401909105014C
:103F000080509C4390F48091020187FF10C086E0AE
:103F100091E00E94571E8091040190910501805804
:103F20009F4F909305018093040110920201BCB849
:103F30005E9BFECF5E9A85B38C2585BB10E00BC0DF
:103F4000DCB85E9BFECF03C0DCB85E9BFECF5E9A02
:103F50001F5F143030F45F9BFECF8CB1843009F0CA
:103F600094CF86E08CB95E9BFECF5E9A112321F040
:103F7000E0E0FCE309950CC0E199FECF8FEF91E002
:103F80009FBB8EBB1DBA0FB6F894E29AE19A0FBEA2
:103F90000E948D1E80E090E01F910F91FF90EF90A6
:0C3FA000DF90CF90BF900895F894FFCF01
:023FAC006400AF
:0400000300003C00BD
:00000001FF
